:0200000001DF1E
:20002300309836C0E0C0D0C298A79930080AB74107200A16D20A8932300A07B70D04C20A08
:20004300D20909430180EAB5010B740171BB90047F716680FED0D0D0E032EAB501012230CC
:2000630099FDC2998A008699C208B60D02D2080A43028022200901220532433280C032A877
:2000830032E6C394304050F5F09402504A752C05D032C0320532433280A832E6C3943040CC
:2000A30036940A5032D52CECD03285F031752C050532433280A832E6C39430C0E0E531750E
:2000C300F005A4252C2432F8D0E0F6D52CE231DE513D5170C20922D032C20922758E0175A9
:2000E3008160758780758922E5B0C454079004C593F58DF58BD28E759852785F760018B802
:2001030001FAD2087A80798071C99103740E71BB748071BB7531021531513D5170E53170B5
:20012300F675A890712D74232531F8A62220020CE531B401037531FF053131BD200614319E
:20014300C5B4090B76000522E522B405EF800204F631BD20071731C5600414F6800D7609AB
:200163000522E522B405EC512A800031BD20040B31C5B409047600803904F620050E31C588
:200183007006E522602C740A14F6702620000AE522B404037522FF0522200109E5227003E8
:2001A300752205152220030A31D27405760018D5E0FA31DE513D5170212774232531F88672
:2001C3002222E53175F005A424332522F8E622E53175F005A424332404F822752C05E5319D
:2001E30075F005A4252C90049493C0E0E53175F005A4252C2432F886F0D0E0B5F003D52CB0
:20020300DD400122752C05E53175F005A4252C90049493C0E0E53175F005A4252C2432F862
:20022300D0E0F6D52CE122E53175F005A42433F8752C05760008D52CFA22E53190048D9393
:20024300C0E071BB31D25166742C719C5166516651665166900488E52293F5F0D0E025F02C
:2002630071BB22E6516B18222430719C22753005E53175F005A425302432F8E6C0E0742A39
:200283002530F8D0E0F6D530E7E52C75F00AA4252BF52BE52E75F00AA4252D75F064A425DE
:2002A3002BF52BE435F0F52C75F010E52FA4F52D75F027E52FA4F52E85F02FE52D252BF515
:2002C3002BE52C352EF52CC2B271089004BDE53193F5907108E52C7E083392B37108C2B27A
:2002E3007108D2B27108DEF1E52B7E083392B37108C2B27108D2B27108DEF17590FF7108F9
:20030300D2B37108227F19DFFE22115D1177E580B4FFF774327F08C0E0115D1177DFFAD0B2
:20032300E0D5E0F1E580B4FFE122710DE580B4FF06115D117780F5F52022B40A00400224B7
:20034300072430719C22C0E054F0C4713DD0E0540F713D2275F00A842430719CE5F024305A
:20036300719C22E4936005719CA380F722F52B936007719CE52BA380F42274C071BB2274C0
:200383000171BB2243A0F0D2A1C2A0D2A2E5A0C2A2D2A2C2A220E7EC22D2A0C0E071AAD01C
:2003A300E0C471AA718722C2A154F053A00F42A0D2A2C2A253A00F22C2A0C0E071AAD0E00D
:2003C300C471AA71872253A00FC2A1C2A0C2A2749671F371FB71FB71FB742071AA71877429
:2003E3002871BB740C71BB740671BB740171BB227F62DFFED5E0F922743071AA743261F34A
:20040300858020300201229004CD7166717D9004DD716674037157712D1203829004E77191
:2004230066717D9004F47166712D1203829005037166717D900FF9E4937149900FF8E4939D
:200443007149712D1203829005127166900FFA9166717D9005197166900FFD9166712D12E6
:20046300038222E4937157742D12039CA3E4937157742D12039CA3E4937157224F7665726D
:20048300666C6F7700050403020080C087C78ECE95D50503050506050305050605030505FD
:2004A3000605030505060503050506050305050605030505060503050506FEFDFBF7EFDF00
:2004C300BF7FFFFEFDFAF4E8D0A0754320436F6E74726F6C20506C75730056657273696FA6
:2004E3006E3A2000436F70797269676874206279004D617274696E20436C617573656E0027
:1D05030053657269616C206E756D6265723A00446174653A200054696D653A2000D7
:080FF8000000000000000000F1
:00000001FF
